:020000040000FA
:0408000061EF09F0AB
:1008100003B26EEF05F0F2B48CEF05F09EB094EFEA
:1008200005F09EB29CEF05F0F2A81AEF04F0F2B2C8
:100830001CEF04F010EF09F0CD90F2929EA026EF8D
:1008400004F00101533F26EF04F0542BB2C1B6F17E
:10085000B3C1B7F1B4C1B8F1B5C1B9F1AEC1B2F12C
:10086000AFC1B3F1B0C1B4F1B1C1B5F1AAC1AEF13C
:10087000ABC1AFF1ACC1B0F1ADC1B1F1A6C1AAF14C
:10088000A7C1ABF1A8C1ACF1A9C1ADF1A2C1A6F15C
:10089000A3C1A7F1A4C1A8F1A5C1A9F19EC1A2F16C
:1008A0009FC1A3F1A0C1A4F1A1C1A5F19AC19EF17C
:1008B0009BC19FF19CC1A0F19DC1A1F1CECF9AF146
:1008C000CFCF9BF153C19CF154C19DF1CF6ACE6A49
:1008D0000101536B546B9E90CD800FBC0F8E0FBAED
:1008E00075EF04F00F8A10EF09F013880F8C0FBE1C
:1008F000B2EF04F09AC19EF19BC19FF19CC1A0F19F
:100900009DC1A1F19EC1A2F19FC1A3F1A0C1A4F11B
:10091000A1C1A5F1A2C1A6F1A3C1A7F1A4C1A8F1EB
:10092000A5C1A9F1A6C1AAF1A7C1ABF1A8C1ACF1BB
:10093000A9C1ADF1AAC1AEF1ABC1AFF1ACC1B0F18B
:10094000ADC1B1F1AEC1B2F1AFC1B3F1B0C1B4F15B
:10095000B1C1B5F1B2C1B6F1B3C1B7F1B4C1B8F12B
:10096000B5C1B9F101015E6B5F6B606B616B9A5150
:100970005E279B515F239C5160239D5161239E51B3
:100980005E279F515F23A0516023A1516123A25193
:100990005E27A3515F23A4516023A5516123A65173
:1009A0005E27A7515F23A8516023A9516123AA5153
:1009B0005E27AB515F23AC516023AD516123AE5133
:1009C0005E27AF515F23B0516023B1516123B25113
:1009D0005E27B3515F23B4516023B5516123B651F3
:1009E0005E27B7515F23B8516023B9516123D89076
:1009F0000101613360335F335E33D89001016133AD
:100A000060335F335E33D8900101613360335F330D
:100A10005E3300C10CF101C10DF102C10EF103C141
:100A20000FF104C110F105C111F106C112F107C1A6
:100A300013F108C114F109C115F10AC116F10BC176
:100A400017F134C135F111B831EF05F00101620E33
:100A5000046F010E056F000E066F000E076F3AEF70
:100A600005F00101A70E046F020E056F000E066F60
:100A7000000E076F5EC100F15FC101F160C102F1BC
:100A800061C103F11BEC20F003BF04D01ABE02D0F9
:100A90001AA0108C11A052EF05F010BA52EF05F019
:100AA0000F80108A0CC100F10DC101F10EC102F1DD
:100AB0000FC103F110C104F111C105F112C106F11A
:100AC00013C107F114C108F115C109F116C10AF1EA
:100AD00017C10BF135C134F110EF09F00392ABB23D
:100AE000AB98AB88030103EE00F080517F0BE92641
:100AF00004C0EFFF802B8151805D700BD8A48B82E6
:100B000000008051815D700BD8A48B9281518019B7
:100B1000D8B4079010EF09F0F2940101453F10EFAF
:100B200009F0462B10EF09F09E900101533F10EFA2
:100B300009F0542B10EF09F09E9213A0C6EF05F0B8
:100B400001015E6B5F6B606B616B626B636B646B0F
:100B5000656B666B676B686B696B536B546BCF6AC5
:100B6000CE6A0F9A0F9C0F9E0101476B486B496B31
:100B70004A6B4B6B4C6B4D6B4E6B4F6B506B516BB1
:100B8000526B456B466BD76AD66A139011B83AEF31
:100B900007F08BB4D3EF05F010ACD3EF05F08B84E6
:100BA000109CD4EF05F08B94C3CF55F1C4CF56F110
:100BB000C28207B443EF06F047C14BF148C14CF184
:100BC00049C14DF14AC14EF15EC162F15FC163F1AD
:100BD00060C164F161C165F113A8F1EF05F0138CF8
:100BE00013989AC1BAF19BC1BBF19CC1BCF19DC1E4
:100BF000BDF19EC1BEF19FC1BFF1A0C1C0F1A1C1B5
:100C0000C1F1A2C1C2F1A3C1C3F1A4C1C4F1A5C184
:100C1000C5F1A6C1C6F1A7C1C7F1A8C1C8F1A9C154
:100C2000C9F1AAC1CAF1ABC1CBF1ACC1CCF1ADC124
:100C3000CDF1AEC1CEF1AFC1CFF1B0C1D0F1B1C1F4
:100C4000D1F1B2C1D2F1B3C1D3F1B4C1D4F1B5C1C4
:100C5000D5F1B6C1D6F1B7C1D7F1B8C1D8F1B9C194
:100C6000D9F1010155515B2756515C23E86A5D2398
:100C70000E2E43EF06F05CC157F15DC158F15B6B7E
:100C80005C6B5D6B078E0201002F10EF09F03C0ECC
:100C9000006F1B50E00BE00AE866128819BE02D014
:100CA00019B4108E00C10CF101C10DF102C10EF199
:100CB00003C10FF104C110F105C111F106C112F118
:100CC00007C113F108C114F109C115F10AC116F1E8
:100CD0000BC117F134C135F101018E6777EF06F0D2
:100CE0008F6777EF06F0906777EF06F091677BEFFD
:100CF00006F0ABEF06F092C100F193C101F194C18F
:100D000002F195C103F10101010E046F000E056FA0
:100D1000000E066F000E076F1BEC20F000C192F171
:100D200001C193F102C194F103C195F10067A0EFF5
:100D300006F00167A0EF06F00267A0EF06F0036778
:100D4000ABEF06F08EC192F18FC193F190C194F197
:100D500091C195F10F80D57ED5BE6ED0D6CF47F12B
:100D6000D7CF48F145C149F1E86AE8CF4AF1138A83
:100D70001ABE02D01AA0108C109047C100F148C1D1
:100D800001F149C102F14AC103F101010A0E046FE8
:100D9000000E056F000E066F000E076F1BEC20F0B3
:100DA00003AF1080010154A7E2EF06F00F9A0F9CE9
:100DB0000F9E0101000E5E6F600E5F6F3D0E606F53
:100DC000080E616F010147BFF2EF06F04867F2EFCE
:100DD00006F04967F2EF06F04A67F2EF06F0F28894
:100DE00017EF07F0F2985E6B5F6B606B616B9A6B4D
:100DF0009B6B9C6B9D6B9E6B9F6BA06BA16BA26BA7
:100E0000A36BA46BA56BA66BA76BA86BA96BAA6B56
:100E1000AB6BAC6BAD6BAE6BAF6BB06BB16BB26B06
:100E2000B36BB46BB56BB66BB76BB86BB96BD76A9A
:100E3000D66A0101456B466B0CC100F10DC101F191
:100E40000EC102F10FC103F110C104F111C105F18E
:100E500012C106F113C107F114C108F115C109F15E
:100E600016C10AF117C10BF135C134F110EF09F0C9
:100E700010EF09F00201002F94EF08F0D59ED6CFB5
:100E800047F1D7CF48F145C149F1E86AE8CF4AF1C7
:100E9000138AD76AD66A0101456B466BD58E1B5003
:100EA000E00BE00AE866128819BE02D019B4108E71
:100EB00018AE1D8C00C10CF101C10DF102C10EF183
:100EC00003C10FF104C110F105C111F106C112F106
:100ED00007C113F108C114F109C115F10AC116F1D6
:100EE0000BC117F134C135F10FA0109A11B884EF7E
:100EF00007F00101620E046F010E056F000E066F10
:100F0000000E076F8DEF07F00101A70E046F020EB0
:100F1000056F000E066F000E076F47C100F148C154
:100F200001F149C102F14AC103F11BEC20F003BFFA
:100F3000A0EF07F01ABE02D01AA0108C11B00F80DB
:100F40000CC100F10DC101F10EC102F10FC103F19D
:100F500010C104F111C105F112C106F113C107F16D
:100F600014C108F115C109F116C10AF117C10BF13D
:100F700035C134F102013C0E006F00C10CF101C11A
:100F80000DF102C10EF103C10FF104C110F105C151
:100F900011F106C112F107C113F108C114F109C121
:100FA00015F10AC116F10BC117F134C135F1010178
:100FB0008E67E2EF07F08F67E2EF07F09067E2EFEE
:100FC00007F09167E6EF07F016EF08F092C100F125
:100FD00093C101F194C102F195C103F10101010E28
:100FE000046F000E056F000E066F000E076F1BECFE
:100FF00020F000C192F101C193F102C194F103C14B
:1010000095F100670BEF08F001670BEF08F002673E
:101010000BEF08F0036716EF08F08EC192F18FC155
:1010200093F190C194F191C195F10F80109047C157
:1010300000F148C101F149C102F14AC103F10101C6
:101040000A0E046F000E056F000E066F000E076F8C
:101050001BEC20F003AF1080010154A73CEF08F017
:101060000F9A0F9C0F9E0101000E5E6F600E5F6F66
:101070003D0E606F080E616F47C100F148C101F17C
:1010800049C102F14AC103F10101140E046F050EBA
:10109000056F000E066F000E076F1BEC20F003AF0C
:1010A00055EF08F0F2887AEF08F0F2985E6B5F6B0C
:1010B000606B616B9A6B9B6B9C6B9D6B9E6B9F6B6C
:1010C000A06BA16BA26BA36BA46BA56BA66BA76BAC
:1010D000A86BA96BAA6BAB6BAC6BAD6BAE6BAF6B5C
:1010E000B06BB16BB26BB36BB46BB56BB66BB76B0C
:1010F000B86BB96B0CC100F10DC101F10EC102F169
:101100000FC103F110C104F111C105F112C106F1C3
:1011100013C107F114C108F115C109F116C10AF193
:1011200017C10BF135C134F18BB49EEF08F010AC50
:101130009EEF08F08B84109C9FEF08F08B94C3CF38
:1011400055F1C4CF56F1C28207B40EEF09F047C182
:101150004BF148C14CF149C14DF14AC14EF15EC15C
:1011600062F15FC163F160C164F161C165F113A80F
:10117000BCEF08F0138C13989AC1BAF19BC1BBF174
:101180009CC1BCF19DC1BDF19EC1BEF19FC1BFF12B
:10119000A0C1C0F1A1C1C1F1A2C1C2F1A3C1C3F1FB
:1011A000A4C1C4F1A5C1C5F1A6C1C6F1A7C1C7F1CB
:1011B000A8C1C8F1A9C1C9F1AAC1CAF1ABC1CBF19B
:1011C000ACC1CCF1ADC1CDF1AEC1CEF1AFC1CFF16B
:1011D000B0C1D0F1B1C1D1F1B2C1D2F1B3C1D3F13B
:1011E000B4C1D4F1B5C1D5F1B6C1D6F1B7C1D7F10B
:1011F000B8C1D8F1B9C1D9F1010155515B27565198
:101200005C23E86A5D230E2E0EEF09F05CC157F1F6
:101210005DC158F15B6B5C6B5D6B078E10EF09F085
:1012200002C0E0FF005001C0D8FF1000A6B216EFC8
:1012300009F00CC0A9FF0BC0A8FFA69EA69CA6841F
:10124000F29E550EA76EAA0EA76EA682F28EA694E7
:10125000A6B228EF09F00C2A1200A96EA69EA69C41
:10126000A680A8500C2A120004012C0E826F41ECBB
:101270000BF016EC21F00C502DEC09F0E8CF00F14A
:101280000C502DEC09F0E8CF01F101AF4DEF09F062
:101290000101FF0E026FFF0E036FB9EC20F029670A
:1012A00059EF09F00401200E826F41EC0BF05EEF64
:1012B00009F004012D0E826F41EC0BF0C3EC1EF01F
:1012C0001200316A076A0F6A106A116A126A136A99
:1012D0000F010E0EC16E860EC06E030EC26E0F01A0
:1012E000896A110E926E080E8A6EF10E936E8B6AE9
:1012F000800E946EF18E8A848B86FC0E2DEC09F0A4
:10130000E8CF0BF00BA011800BA211820BA411846B
:101310000BA81188C90E2DEC09F0E8CF18F0CA0E01
:101320002DEC09F0E8CF19F0CB0E2DEC09F0E8CF49
:101330001AF0CC0E2DEC09F0E8CF1BF0CE0E2DEC00
:1013400009F0E8CF14F0CD0E2DEC09F0E8CF30F025
:101350001D6A1E6A0E6A01015B6B5C6B5D6B576BED
:10136000586BF29A0101476B486B496B4A6B4B6BA8
:101370004C6B4D6B4E6B4F6B506B516B526B456BA7
:10138000466BD76AD66A0F01280ED56EF28A9D90F9
:10139000B00ECD6E01015E6B5F6B606B616B626B5B
:1013A000636B646B656B666B676B686B696B536BC8
:1013B000546BCF6ACE6A0F9A0F9C0F9E9D80760E5B
:1013C000CA6E9D8202013C0E006FCC6A160E2DEC97
:1013D00009F0E8CF00F1170E2DEC09F0E8CF01F18C
:1013E000180E2DEC09F0E8CF02F1190E2DEC09F0E2
:1013F000E8CF03F1010103AF18EF0AF016EC21F07A
:10140000160E0C6E00C10BF016EC09F0170E0C6EE8
:1014100001C10BF016EC09F0180E0C6E02C10BF0B6
:1014200016EC09F0190E0C6E03C10BF016EC09F066
:1014300000C18EF101C18FF102C190F103C191F1A0
:1014400000C192F101C193F102C194F103C195F180
:101450001A0E2DEC09F0E8CF00F11B0E2DEC09F06F
:10146000E8CF01F11C0E2DEC09F0E8CF02F11D0EC2
:101470002DEC09F0E8CF03F1010103AF6EEF0AF0A4
:1014800016EC21F01A0E0C6E00C10BF016EC09F0F0
:101490001B0E0C6E01C10BF016EC09F01C0E0C6E4D
:1014A00002C10BF016EC09F01D0E0C6E03C10BF01F
:1014B00016EC09F01A0E2DEC09F0E8CF00F11B0E26
:1014C0002DEC09F0E8CF01F11C0E2DEC09F0E8CF6E
:1014D00002F11D0E2DEC09F0E8CF03F100C196F1E9
:1014E00001C197F102C198F103C199F1240EAC6ECC
:1014F000900EAB6E240EAC6E080EB86E000EB06E81
:101500001F0EAF6E0401806B816B0F01900EAB6EEE
:101510000F019D8A0301806B816BC26B8B920790D8
:101520000001F28EF28C07B071EF1DF00FB069EF81
:1015300016F010BE69EF16F012B869EF16F003014D
:10154000805181197F0BD8B471EF1DF013EE00F0BC
:1015500081517F0BE126812BE7CFE8FFE00BD8B468
:1015600071EF1DF023EE82F0C2513F0BD926E7CF79
:10157000DFFFC22BDF50780AD8A471EF1DF007807F
:1015800092C100F193C101F194C102F195C103F13F
:101590000101040E046F000E056F000E066F000EB1
:1015A000076F1BEC20F000AFDFEF0AF00101030E24
:1015B000926F000E936F000E946F000E956F0301F3
:1015C0008251720AD8B445EF16F08251520AD8B44B
:1015D00045EF16F08251750AD8B445EF16F08251E6
:1015E000630AD8B42BEF1AF08251690AD8B4EFEF2E
:1015F00012F082517A0AD8B402EF14F08251490AEB
:10160000D8B414EF12F08251500AD8B432EF11F06E
:101610008251700AD8B475EF11F08251540AD8B4CF
:10162000A0EF11F08251740AD8B4E6EF11F08251A4
:10163000410AD8B457EF0CF082514B0AD8B455EF99
:101640000BF082516D0AD8B48AEF10F082514D0A26
:10165000D8B4A3EF10F08251730AD8B475EF15F027
:101660008251530AD8B4DAEF15F08251660AD8B421
:1016700075EF12F08251590AD8B4DBEF0FF062EF28
:101680001AF0040114EE00F080517F0BE12682C4B1
:10169000E7FF802B120004010D0E826F41EC0BF06E
:1016A0000A0E826F41EC0BF0120004014B0E826FA8
:1016B00041EC0BF004012C0E826F41EC0BF081B871
:1016C00002D030B630D003018351430AD8B49AEF28
:1016D0000BF003018351630AD8B49CEF0BF00301B4
:1016E0008351520AD8B49EEF0BF003018351720A62
:1016F000D8B4A0EF0BF003018351470AD8B4A2EF8E
:101700000BF003018351670AD8B4A4EF0BF0030177
:101710008351540AD8B4A6EF0BF003018351740A25
:10172000D8B415EF0CF003018351550AD8B4A8EFD3
:101730000BF082D030807AD0309078D0308276D062
:10174000309274D0308472D0309470D030866ED0A5
:1017500084C330F185C331F186C332F187C333F1DD
:101760000101296B64EC21F0DBEC20F000C104F1F5
:1017700001C105F102C106F103C107F157EC21F0E7
:10178000200EF86EF76AF66A0900F5CF2CF1090011
:10179000F5CF2DF10900F5CF2EF10900F5CF2FF18E
:1017A0000900F5CF30F10900F5CF31F10900F5CF8F
:1017B00032F10900F5CF33F10101296B64EC21F01E
:1017C000DBEC20F01BEC20F00067EEEF0BF0016784
:1017D000EEEF0BF00267EEEF0BF0036701D025D0C0
:1017E00004014E0E826F41EC0BF004016F0E826F0C
:1017F00041EC0BF004014D0E826F41EC0BF0040143
:10180000610E826F41EC0BF00401740E826F41ECAB
:101810000BF00401630E826F41EC0BF00401680EC3
:10182000826F41EC0BF060EF1AF03096CD0E0C6E2B
:1018300030C00BF016EC09F0CD0E2DEC09F0E8CF1E
:1018400030F030B006D00401630E826F41EC0BF033
:1018500005D00401430E826F41EC0BF030B206D08C
:101860000401720E826F41EC0BF005D00401520EA0
:10187000826F41EC0BF030B406D00401670E826F2A
:1018800041EC0BF005D00401470E826F41EC0BF0E8
:1018900030B606D00401740E826F41EC0BF005D017
:1018A0000401540E826F41EC0BF060EF1AF004015A
:1018B000410E826F41EC0BF003018351310AD8B421
:1018C000FBEF0EF003018351320AD8B42BEF0EF078
:1018D00003018351330AD8B4B4EF0DF003018351EF
:1018E000340AD8B4A4EF0CF003018351350AD8B4FC
:1018F00081EF0CF004013F0E826F41EC0BF060EFC2
:101900001AF004012C0E826F41EC0BF0030184519C
:10191000300AD8B494EF0CF003018451310AD8B4E2
:101920009CEF0CF0EDEF0DF08B900401300E826F08
:1019300041EC0BF0A2EF0CF08B800401310E826FB2
:1019400041EC0BF060EF1AF0CC0E2DEC09F0E8CF73
:101950000BF004012C0E826F41EC0BF0030184515B
:10196000310AD8B4C8EF0CF003018451300AD8B45E
:10197000CAEF0CF0030184514D0AD8B4D4EF0CF037
:1019800003018451540AD8B4DBEF0CF0F2EF0CF0F1
:101990008A8401D08A940BAE04D00BAC02D00BBA6F
:1019A00021D0E00E0B1218D01F0E0B168539E8441B
:1019B000E00B0B1211D0E00E0B1657EC21F085C393
:1019C00032F186C333F10101296B64EC21F0DBECC9
:1019D00020F000511F0B0B12CC0E0C6E0BC00BF045
:1019E00016EC09F00401340E826F41EC0BF0040197
:1019F0002C0E826F41EC0BF0CC0E2DEC09F0E8CFF1
:101A00001BF08AB406D00401300E826F41EC0BF05B
:101A100005D00401310E826F41EC0BF004012C0E55
:101A2000826F41EC0BF01B38E840070BE8CF82F4E3
:101A30000401300E822741EC0BF004012C0E826F62
:101A400041EC0BF016EC21F01B501F0BE8CF00F11E
:101A5000B9EC20F032C182F40401300E822741EC4F
:101A60000BF033C182F40401300E822741EC0BF0FD
:101A700004012C0E826F41EC0BF016EC21F02EC00D
:101A800000F100AF0BD0FF0E016FFF0E026FFF0ED3
:101A9000036F04012D0E826F41EC0BF0B9EC20F0C6
:101AA00031C182F40401300E822741EC0BF032C1C7
:101AB00082F40401300E822741EC0BF033C182F432
:101AC0000401300E822741EC0BF004012C0E826FD2
:101AD00041EC0BF016EC21F02DC000F1B9EC20F038
:101AE00031C182F40401300E822741EC0BF032C187
:101AF00082F40401300E822741EC0BF033C182F4F2
:101B00000401300E822741EC0BF004012C0E826F91
:101B100041EC0BF016EC21F02FC000F100AF0BD020
:101B2000FF0E016FFF0E026FFF0E036F04012D0EFB
:101B3000826F41EC0BF0B9EC20F031C182F404016A
:101B4000300E822741EC0BF032C182F40401300EDA
:101B5000822741EC0BF033C182F40401300E82275E
:101B600041EC0BF060EF1AF0CB0E2DEC09F0E8CF52
:101B70000BF004012C0E826F41EC0BF00301845139
:101B8000450AD8B4D8EF0DF003018451440AD8B403
:101B9000DBEF0DF003018451300AD8B4DEEF0DF015
:101BA00003018451310AD8B4E2EF0DF0EDEF0DF0EE
:101BB0000B9EE7EF0DF00B8EE7EF0DF0FC0E0B1612
:101BC000E7EF0DF0FC0E0B160B80E7EF0DF0CB0EE0
:101BD0000C6E0BC00BF016EC09F00401330E826F93
:101BE00041EC0BF004012C0E826F41EC0BF0CB0E9C
:101BF0002DEC09F0E8CF1AF01ABE06EF0EF0040142
:101C0000450E826F41EC0BF00BEF0EF00401440E19
:101C1000826F41EC0BF004012C0E826F41EC0BF053
:101C20000401300E826F41EC0BF004012C0E826F28
:101C300041EC0BF01AB024EF0EF00401300E826F6D
:101C400041EC0BF029EF0EF00401310E826F41ECF4
:101C50000BF060EF1AF0CA0E2DEC09F0E8CF0BF094
:101C600004012C0E826F41EC0BF003018451450AF4
:101C7000D8B467EF0EF003018451440AD8B46AEF78
:101C80000EF0030184514D0AD8B473EF0EF0030136
:101C90008451410AD8B46DEF0EF003018451460A15
:101CA000D8B470EF0EF003018451560AD8B47BEF1C
:101CB0000EF003018451500AD8B486EF0EF00301F0
:101CC0008451520AD8B489EF0EF092EF0EF00B9EB9
:101CD0008CEF0EF00B8E8CEF0EF00B9C8CEF0EF059
:101CE0000B8C8CEF0EF0FC0E0B1685C3E8FF030B7C
:101CF0000B128CEF0EF0C70E0B1685C3E8FF070B17
:101D0000E846E846E8460B128CEF0EF00B848CEFA9
:101D10000EF00B948CEF0EF0CA0E0C6E0BC00BF095
:101D200016EC09F0CA0E2DEC09F0E8CF19F0040109
:101D3000320E826F41EC0BF004012C0E826F41ECED
:101D40000BF019BEABEF0EF00401450E826F41ECB3
:101D50000BF0B0EF0EF00401440E826F41EC0BF07B
:101D600004012C0E826F41EC0BF019C0E8FF030B4D
:101D7000E8CF82F40401300E822741EC0BF004011D
:101D80002C0E826F41EC0BF019BCCEEF0EF004016B
:101D9000410E826F41EC0BF0D3EF0EF00401460EC2
:101DA000826F41EC0BF004012C0E826F41EC0BF0C2
:101DB00019C0E8FF380BE842E842E842E8CF82F475
:101DC0000401300E822741EC0BF004012C0E826FCF
:101DD00041EC0BF019B4F4EF0EF00401520E826FD7
:101DE00041EC0BF0F9EF0EF00401500E826F41EC64
:101DF0000BF060EF1AF0C90E2DEC09F0E8CF0BF0F4
:101E000004012C0E826F41EC0BF003018451450A52
:101E1000D8B419EF0FF003018451440AD8B41CEF71
:101E20000FF0030184514D0AD8B41FEF0FF02DEFCE
:101E30000FF00B9E27EF0FF00B8E27EF0FF0F80E31
:101E40000B1685C3E8FF070B0B1227EF0FF0C90E27
:101E50000C6E0BC00BF016EC09F00401310E826F12
:101E600041EC0BF004012C0E826F41EC0BF0C90E1B
:101E70002DEC09F0E8CF18F018BE06D00401450E8D
:101E8000826F41EC0BF005D00401440E826F41ECEF
:101E90000BF004012C0E826F41EC0BF018C0E8FF30
:101EA000070BE8CF82F40401300E822741EC0BF0DF
:101EB00004012C0E826F41EC0BF0078016EC21F030
:101EC00029C0E8FF003B00430043030BB9EC20F0BE
:101ED00033C182F40401300E822741EC0BF004017F
:101EE0002C0E826F41EC0BF016EC21F029C001F1B1
:101EF000019F019D2AC000F10101B9EC20F02FC122
:101F000082F40401300E822741EC0BF030C182F4E0
:101F10000401300E822741EC0BF031C182F4040140
:101F2000300E822741EC0BF032C182F40401300EF6
:101F3000822741EC0BF033C182F40401300E82277A
:101F400041EC0BF004012C0E826F41EC0BF016EC0F
:101F500021F02BC001F12CC000F1D89001330033E7
:101F6000D890013300330101B9EC20F02FC182F485
:101F70000401300E822741EC0BF030C182F40401E1
:101F8000300E822741EC0BF031C182F40401300E97
:101F9000822741EC0BF032C182F40401300E82271B
:101FA00041EC0BF033C182F40401300E822741EC86
:101FB0000BF060EF1AF0FC0E2DEC09F0E8CF0BF0FF
:101FC00003018351520AD8B412EF10F00301835178
:101FD000720AD8B415EF10F003018351500AD8B437
:101FE00018EF10F003018351700AD8B41BEF10F002
:101FF00003018351550AD8B41EEF10F00301835139
:10200000750AD8B421EF10F003018351430AD8B404
:102010002AEF10F003018351630AD8B42DEF10F0BA
:1020200036EF10F00B9030EF10F00B8030EF10F027
:102030000B9230EF10F00B8230EF10F00B9430EF7A
:1020400010F00B8430EF10F00B9630EF10F00B8691
:1020500030EF10F00B9830EF10F00B8830EF10F0ED
:10206000FC0E0C6E0BC00BF016EC09F00401590EBF
:10207000826F41EC0BF01190119211941198FC0EAB
:102080002DEC09F0E8CF0BF00BA011800BA2118210
:102090000BA411840BA8118811A056EF10F00401B5
:1020A000520E826F41EC0BF05BEF10F00401720EE8
:1020B000826F41EC0BF011A865EF10F00401430EA4
:1020C000826F41EC0BF06AEF10F00401630E826F37
:1020D00041EC0BF011A274EF10F00401500E826F6E
:1020E00041EC0BF079EF10F00401700E826F41ECBF
:1020F0000BF011A483EF10F00401550E826F41EC38
:102100000BF088EF10F00401750E826F41EC0BF0BC
:1021100060EF1AF004016D0E826F41EC0BF00301C9
:102120008351300AD8B4E2EF10F003018351310A31
:10213000D8B4F5EF10F003018351320AD8B408EF98
:1021400011F062EF1AF004014D0E826F41EC0BF0BA
:1021500057EC21F084C331F185C332F186C333F1EA
:102160000101296B64EC21F0DBEC20F003018351C9
:10217000300AD8B4CAEF10F003018351310AD8B441
:10218000D2EF10F003018351320AD8B4DAEF10F025
:1021900062EF1AF0FD0E0C6E00C10BF016EC09F0A8
:1021A000E2EF10F0FE0E0C6E00C10BF016EC09F021
:1021B000F5EF10F0FF0E0C6E00C10BF016EC09F0FD
:1021C00008EF11F00401300E826F41EC0BF00401B6
:1021D0002C0E826F41EC0BF016EC21F0FD0E2DEC75
:1021E00009F0E8CF00F119EF11F00401310E826F10
:1021F00041EC0BF004012C0E826F41EC0BF016EC5D
:1022000021F0FE0E2DEC09F0E8CF00F119EF11F0EE
:102210000401320E826F41EC0BF016EC21F0040148
:102220002C0E826F41EC0BF0FF0E2DEC09F0E8CF85
:1022300000F1B9EC20F031C182F40401300E8227A4
:1022400041EC0BF032C182F40401300E822741ECE4
:102250000BF033C182F40401300E822741EC0BF005
:1022600060EF1AF083C32AF184C32BF185C32CF1EC
:1022700086C32DF187C32EF188C32FF189C330F1B6
:102280008AC331F18BC332F18CC333F1010164ECA9
:1022900021F0DBEC20F0160E0C6E00C10BF016ECFA
:1022A00009F0170E0C6E01C10BF016EC09F0180EB8
:1022B0000C6E02C10BF016EC09F0190E0C6E03C186
:1022C0000BF016EC09F000C18EF101C18FF102C1D3
:1022D00090F103C191F100C192F101C193F102C1EA
:1022E00094F103C195F114EF12F083C32AF184C372
:1022F0002BF185C32CF186C32DF187C32EF188C342
:102300002FF189C330F18AC331F18BC332F18CC311
:1023100033F1010164EC21F0DBEC20F000C18EF11F
:1023200001C18FF102C190F103C191F100C192F19D
:1023300001C193F102C194F103C195F114EF12F0C0
:1023400083C32AF184C32BF185C32CF186C32DF1FD
:1023500087C32EF188C32FF189C330F18AC331F1CD
:102360008CC332F18DC333F1010164EC21F0DBEC5D
:1023700020F00101000E046F000E056F010E066FC4
:10238000000E076F2CEC20F01A0E0C6E00C10BF043
:1023900016EC09F01B0E0C6E01C10BF016EC09F0E7
:1023A0001C0E0C6E02C10BF016EC09F01D0E0C6E2B
:1023B00003C10BF016EC09F000C196F101C197F1D1
:1023C00002C198F103C199F114EF12F083C32AF10D
:1023D00084C32BF185C32CF186C32DF187C32EF165
:1023E00088C32FF189C330F18AC331F18CC332F134
:1023F0008DC333F1010164EC21F0DBEC20F001012D
:10240000000E046F000E056F010E066F000E076FC1
:102410002CEC20F000C196F101C197F102C198F1B6
:1024200003C199F114EF12F0160E2DEC09F0E8CF6C
:1024300000F1170E2DEC09F0E8CF01F1180E2DEC8C
:1024400009F0E8CF02F1190E2DEC09F0E8CF03F105
:10245000B9EC20F07CEC1EF00401730E826F41ECAD
:102460000BF004012C0E826F41EC0BF08EC100F1D9
:102470008FC101F190C102F191C103F1B9EC20F0DB
:102480007CEC1EF00401730E826F41EC0BF0040132
:102490002C0E826F41EC0BF01A0E2DEC09F0E8CFF8
:1024A00000F11B0E2DEC09F0E8CF01F11C0E2DEC14
:1024B00009F0E8CF02F11D0E2DEC09F0E8CF03F191
:1024C0007DEC1AF004012C0E826F41EC0BF096C1EA
:1024D00000F197C101F198C102F199C103F17DECBE
:1024E0001AF04BEC0BF062EF1AF00401660E826FEB
:1024F00041EC0BF003018351780AD8B4A2EF12F03B
:1025000003018351430AD8B4A6EF12F003018351AB
:10251000460AD8B4AFEF12F0030183B102D08B9614
:1025200001D08B8683B302D08A9401D08A8484B18F
:1025300002D08B9A01D08B8A84B302D08B9801D0C1
:102540008B881380B2EC12F060EF1AF0149ECE0E5E
:102550000C6E14C00BF016EC09F0A2EF12F0148E02
:10256000A7EF12F004012C0E826F41EC0BF0300E3D
:102570008BB602D0E89001D0E8808AB402D0E8920D
:1025800001D0E882E8CF82F441EC0BF004012C0E7C
:10259000826F41EC0BF0300E8BBA02D0E89001D084
:1025A000E8808BB802D0E89201D0E882E8CF82F4CC
:1025B00041EC0BF004012C0E826F41EC0BF014AED9
:1025C000E9EF12F00401460E826F41EC0BF0EEEFE2
:1025D00012F00401430E826F41EC0BF01200040173
:1025E000690E826F41EC0BF004012C0E826F41ECFE
:1025F0000BF00101040E006F000E016F000E026F60
:10260000000E036FB9EC20F02CC182F40401300EEF
:10261000822741EC0BF02DC182F40401300E822799
:1026200041EC0BF02EC182F40401300E822741EC04
:102630000BF02FC182F40401300E822741EC0BF025
:1026400030C182F40401300E822741EC0BF031C11D
:1026500082F40401300E822741EC0BF032C182F487
:102660000401300E822741EC0BF033C182F40401E7
:10267000300E822741EC0BF004012C0E826F41ECEE
:102680000BF00101040E006F000E016F000E026FCF
:10269000000E036FB9EC20F02CC182F40401300E5F
:1026A000822741EC0BF02DC182F40401300E822709
:1026B00041EC0BF02EC182F40401300E822741EC74
:1026C0000BF02FC182F40401300E822741EC0BF095
:1026D00030C182F40401300E822741EC0BF031C18D
:1026E00082F40401300E822741EC0BF032C182F4F7
:1026F0000401300E822741EC0BF033C182F4040157
:10270000300E822741EC0BF004012C0E826F41EC5D
:102710000BF001013B0E006F000E016F000E026F07
:10272000000E036FB9EC20F02CC182F40401300ECE
:10273000822741EC0BF02DC182F40401300E822778
:1027400041EC0BF02EC182F40401300E822741ECE3
:102750000BF02FC182F40401300E822741EC0BF004
:1027600030C182F40401300E822741EC0BF031C1FC
:1027700082F40401300E822741EC0BF032C182F466
:102780000401300E822741EC0BF033C182F40401C6
:10279000300E822741EC0BF004012C0E826F41ECCD
:1027A0000BF0200EF86EF76AF66A04010900F5CF07
:1027B00082F441EC0BF00900F5CF82F441EC0BF010
:1027C0000900F5CF82F441EC0BF00900F5CF82F45B
:1027D00041EC0BF00900F5CF82F441EC0BF009005D
:1027E000F5CF82F441EC0BF00900F5CF82F441EC17
:1027F0000BF00900F5CF82F441EC0BF04BEC0BF041
:1028000062EF1AF08351630AD8A460EF1AF0845182
:10281000610AD8A460EF1AF085516C0AD8A460EF61
:102820001AF08651410A3FE08651440A1BE0865166
:10283000420AD8B466EF14F08651350AD8B4ECEFEA
:102840001BF08651360AD8B441EF1CF08651370A86
:10285000D8B4AAEF1CF08651380AD8B408EF1DF09E
:1028600060EF1AF00798079A04017A0E826F41EC24
:102870000BF00401780E826F41EC0BF00401640E42
:10288000826F41EC0BF00401550E826F41EC0BF0AE
:102890004FEF14F004014C0E826F41EC0BF04BEC47
:1028A0000BF062EF1AF00788079A04017A0E826F24
:1028B00041EC0BF00401410E826F41EC0BF004017E
:1028C000610E826F41EC0BF043EF14F00798078A1A
:1028D00004017A0E826F41EC0BF00401420E826F0C
:1028E00041EC0BF00401610E826F41EC0BF043EF01
:1028F00014F00101666784EF14F0676784EF14F049
:10290000686784EF14F0696715D04F678FEF14F094
:1029100050678FEF14F051678FEF14F052670AD0B1
:102920000101000E006F000E016F000E026F000E1D
:10293000036F120011B80AD00101620E046F010E7C
:10294000056F000E066F000E076F09D00101A70E7C
:10295000046F020E056F000E066F000E076F66C152
:1029600000F167C101F168C102F169C103F11BEC1B
:1029700020F003BF2CEF15F0119A119C0101000EFD
:10298000046FA80E056F550E066F020E076F66C125
:1029900000F167C101F168C102F169C103F166C1CB
:1029A0008AF167C18BF168C18CF169C18DF11BECB3
:1029B00020F003BF0BD00101000E8A6FA80E8B6FB1
:1029C000550E8C6F020E8D6F118A119C0E0E2DEC20
:1029D00009F0E8CF18F10F0E2DEC09F0E8CF19F14E
:1029E000100E2DEC09F0E8CF1AF1110E2DEC09F0C4
:1029F000E8CF1BF164EC1FF08AC104F18BC105F133
:102A00008CC106F18DC107F11BEC20F0078228EC88
:102A10001FF064EC1FF0079228EC1FF08AC100F150
:102A20008BC101F18CC102F18DC103F1079228EC39
:102A30001FF0CC0E046FE00E056F870E066F050EBB
:102A4000076F1BEC20F000C118F101C119F102C1A0
:102A50001AF103C11BF140D013AA31EF15F0138E08
:102A6000139A119C119A0101800E006F1A0E016FCA
:102A7000060E026F000E036F4FC104F150C105F145
:102A800051C106F152C107F11BEC20F003AF05D094
:102A900016EC21F0118C119A12000E0E2DEC09F09B
:102AA000E8CF18F10F0E2DEC09F0E8CF19F1100E58
:102AB0002DEC09F0E8CF1AF1110E2DEC09F0E8CF5A
:102AC0001BF14FC100F150C101F151C102F152C1DE
:102AD00003F1078228EC1FF018C100F119C101F1C0
:102AE0001AC102F11BC103F112000401730E826FBF
:102AF00041EC0BF004012C0E826F41EC0BF00784CB
:102B000062C166F163C167F164C168F165C169F1D1
:102B10004BC14FF14CC150F14DC151F14EC152F179
:102B200057C159F158C15AF107949BEC15F04BEC81
:102B30000BF062EF1AF066C100F167C101F168C1E4
:102B400002F169C103F10101B9EC20F07CEC1EF047
:102B50000401630E826F41EC0BF004012C0E826FB6
:102B600041EC0BF04FC100F150C101F151C102F134
:102B700052C103F10101B9EC20F07CEC1EF004011C
:102B8000660E826F41EC0BF004012C0E826F41EC5B
:102B90000BF016EC21F059C100F15AC101F101010D
:102BA000B9EC20F07CEC1EF00401740E826F41EC55
:102BB0000BF0120010820401530E826F41EC0BF0F7
:102BC00004012C0E826F41EC0BF083C32AF184C305
:102BD0002BF185C32CF186C32DF187C32EF188C359
:102BE0002FF189C330F18AC331F18BC332F18CC329
:102BF00033F1010164EC21F0DBEC20F000C166F15F
:102C000001C167F102C168F103C169F18EC32AF104
:102C10008FC32BF190C32CF191C32DF192C32EF1F0
:102C200093C32FF194C330F195C331F196C332F1C0
:102C300097C333F1010164EC21F0DBEC20F000C11B
:102C40004FF101C150F102C151F103C152F157ECF2
:102C500021F099C32FF19AC330F19BC331F19CC38A
:102C600032F19DC333F1010164EC21F0DBEC20F083
:102C700000C159F101C15AF19BEC15F004012C0E71
:102C8000826F41EC0BF055EF16F0118E1AA002D0B6
:102C90001AAE108C19BE02D019A4108E03018251F5
:102CA000520A02E10F8201D00F928251750A02E1AD
:102CB000108401D010948251550A02E1108601D08F
:102CC00010968351310A03E11382138402D01392C8
:102CD000139411A003D011A401D01084078410B262
:102CE000D3EF16F010A4B7EF16F0BAC166F1BBC16E
:102CF00067F1BCC168F1BDC169F1BEC16AF1BFC174
:102D00006BF1C0C16CF1C1C16DF1C2C16EF1C3C143
:102D10006FF1C4C170F1C5C171F1C6C172F1C7C113
:102D200073F1C8C174F1C9C175F1CAC176F1CBC1E3
:102D300077F1CCC178F1CDC179F1CEC17AF1CFC1B3
:102D40007BF1D0C17CF1D1C17DF1D2C17EF1D3C183
:102D50007FF1D4C180F1D5C181F1D6C182F1D7C153
:102D600083F1D8C184F1D9C185F1BFEF16F062C1FA
:102D700066F163C167F164C168F165C169F1BAC107
:102D800086F1BBC187F1BCC188F1BDC189F14BC1DE
:102D90004FF14CC150F14DC151F14EC152F157C1EB
:102DA00059F158C15AF107940FA0F5EF16F001013F
:102DB0009667E2EF16F09767E2EF16F09867E2EF9A
:102DC00016F09967E6EF16F0F5EF16F079EC14F0CF
:102DD00096C104F197C105F198C106F199C107F1B7
:102DE0001BEC20F003BF26EF1AF079EC14F0010180
:102DF000000E046F000E056F010E066F000E076FC8
:102E00004CEC20F011A02AD011A228D0B9EC20F06F
:102E1000296701D005D004012D0E826F41EC0BF023
:102E200030C182F40401300E822741EC0BF031C135
:102E300082F40401300E822741EC0BF032C182F49F
:102E40000401300E822741EC0BF033C182F40401FF
:102E5000300E822741EC0BF04BEC0BF012A8C5D0E2
:102E600012981BC01CF01C3A1C42070E1C160001D5
:102E70001C50000AD8B4C1EF17F000011C50010A21
:102E8000D8B44DEF17F000011C50020AD8B44BEF34
:102E900017F0F3EF17F0F3EF17F016EC21F02BC05B
:102EA00001F12CC000F1D89001330033D8900133E8
:102EB00000330101630E046F000E056F000E066FF4
:102EC000000E076F4CEC20F0280E046F000E056F0B
:102ED000000E066F000E076F1BEC20F000C12EF0F5
:102EE00016EC21F029C001F1019F019D2AC000F1DB
:102EF0000101A40E046F000E056F000E066F000E98
:102F0000076F4CEC20F000C12DF000C104F101C1AD
:102F100005F102C106F103C107F1640E006F000E56
:102F2000016F000E026F000E036F1BEC20F0050E08
:102F3000046F000E056F000E066F000E076F4CEC5D
:102F400020F000C104F101C105F102C106F103C185
:102F500007F116EC21F02EC000F11BEC20F000C1AF
:102F60002FF02FC0E8FF050F2E5C03E78A84F3EFF4
:102F700017F02FC0E8FF0A0F2E5C01E68A94F3EFEA
:102F800017F000C124F101C125F102C126F103C1EE
:102F900027F116EC21F01CEC21F01B501F0BE8CFA1
:102FA00000F10101640E046F000E056F000E066F44
:102FB000000E076F2CEC20F024C104F125C105F1AF
:102FC00026C106F127C107F11BEC20F003BF02D098
:102FD0008A9401D08A8424C100F125C101F126C15F
:102FE00002F127C103F162EF1AF000C124F101C11F
:102FF00025F102C126F103C127F110AE4DD0109E7C
:1030000000C108F101C109F102C10AF103C10BF1CC
:10301000B9EC20F030C1DAF131C1DBF132C1DCF1C1
:1030200033C1DDF108C100F109C101F10AC102F1AA
:103030000BC103F101016C0E046F070E056F000E4A
:10304000066F000E076F1BEC20F003BF04D00101D8
:10305000550EDE6F1CD008C100F109C101F10AC193
:1030600002F10BC103F10101A40E046F060E056FFE
:10307000000E066F000E076F1BEC20F003BF04D09C
:1030800001017F0EDE6F03D00101FF0EDE6F1D8E8A
:1030900011AE26EF1AF0119E24C100F125C101F1F5
:1030A00026C102F127C103F111A005D011A203D05E
:1030B0000FB026EF1AF010A465EF18F00401750E9A
:1030C000826F41EC0BF06AEF18F00401720E826F10
:1030D00041EC0BF004012C0E826F41EC0BF0B9ECCB
:1030E00020F0296779EF18F00401200E826F7CEF41
:1030F00018F004012D0E826F41EC0BF030C182F408
:103100000401300E822741EC0BF031C182F404013E
:10311000300E822741EC0BF004012E0E826F41EC41
:103120000BF032C182F40401300E822741EC0BF027
:1031300033C182F40401300E822741EC0BF004010C
:103140006D0E826F41EC0BF004012C0E826F41EC8E
:103150000BF04FC100F150C101F151C102F152C158
:1031600003F10101B9EC20F07CEC1EF00401480EE3
:10317000826F41EC0BF004017A0E826F41EC0BF090
:1031800004012C0E826F41EC0BF066C100F167C1A7
:1031900001F168C102F169C103F10101B9EC20F04C
:1031A0007CEC1EF00401630E826F41EC0BF0040115
:1031B0002C0E826F41EC0BF066C100F167C101F18A
:1031C00068C102F169C103F101010A0E046F000E2A
:1031D000056F000E066F000E076F2CEC20F0000E3E
:1031E000046F120E056F000E066F000E076F4CEC99
:1031F00020F0B9EC20F02AC182F40401300E8227BD
:1032000041EC0BF02BC182F40401300E822741EC1B
:103210000BF02CC182F40401300E822741EC0BF03C
:103220002DC182F40401300E822741EC0BF02EC137
:1032300082F40401300E822741EC0BF02FC182F49E
:103240000401300E822741EC0BF030C182F40401FE
:10325000300E822741EC0BF004012E0E826F41EC00
:103260000BF031C182F40401300E822741EC0BF0E7
:1032700032C182F40401300E822741EC0BF033C1DD
:1032800082F40401300E822741EC0BF00401730E2E
:10329000826F41EC0BF004012C0E826F41EC0BF0BD
:1032A00016EC21F059C100F15AC101F18CEC1BF070
:1032B000B2EC12F014BE73EF19F08BBA02D0E890A2
:1032C00001D0E8808BB802D0E89201D0E882E82AE9
:1032D000030BE8B002D08B9A01D08B8AE8B202D0FF
:1032E0008B9801D08B8813A2C5EF19F004012C0E26
:1032F000826F41EC0BF086C166F187C167F188C12E
:1033000068F189C169F179EC14F00101000E046FD4
:10331000000E056F010E066F000E076F4CEC20F0DB
:10332000B9EC20F029679AEF19F00401200E826FA2
:103330009DEF19F004012D0E826F41EC0BF030C1AE
:1033400082F40401300E822741EC0BF031C182F48B
:103350000401300E822741EC0BF004012E0E826F27
:1033600041EC0BF032C182F40401300E822741ECB3
:103370000BF033C182F40401300E822741EC0BF0D4
:1033800004016D0E826F41EC0BF013A4ECEF19F009
:1033900004012C0E826F41EC0BF013ACDAEF19F044
:1033A0000401500E826F41EC0BF0139C1398139A9A
:1033B000ECEF19F013AEE7EF19F00401460E826F3F
:1033C00041EC0BF0139E1398139AECEF19F00401E3
:1033D000530E826F41EC0BF00FB2F2EF19F00FA019
:1033E00024EF1AF004012C0E826F41EC0BF0200E3A
:1033F000F86EF76AF66A04010900F5CF82F441EC31
:103400000BF00900F5CF82F441EC0BF00900F5CF89
:1034100082F441EC0BF00900F5CF82F441EC0BF0A3
:103420000900F5CF82F441EC0BF00900F5CF82F4EE
:1034300041EC0BF00900F5CF82F441EC0BF00900F0
:10344000F5CF82F441EC0BF04BEC0BF00F90109E9B
:10345000129862EF1AF00401630E826F41EC0BF0D8
:1034600004012C0E826F41EC0BF068EC1AF00401A1
:103470002C0E826F41EC0BF0DBEC1AF004012C0EE9
:10348000826F41EC0BF057EC1BF004012C0E826FA5
:1034900041EC0BF00101F80E006FCD0E016F660ECE
:1034A000026F030E036F7DEC1AF004012C0E826F85
:1034B00041EC0BF06DEC1BF04BEC0BF062EF1AF0F3
:1034C0004BEC0BF00301C26B0790109271EF1DF0F3
:1034D000D8900E0E2DEC09F0E8CF00F10F0E2DEC78
:1034E00009F0E8CF01F1100E2DEC09F0E8CF02F160
:1034F000110E2DEC09F0E8CF03F10101000E046F6D
:10350000000E056F010E066F000E076F4CEC20F0E9
:10351000B9EC20F02AC182F40401300E822741EC7C
:103520000BF02BC182F40401300E822741EC0BF02A
:103530002CC182F40401300E822741EC0BF02DC126
:1035400082F40401300E822741EC0BF02EC182F48C
:103550000401300E822741EC0BF02FC182F40401EC
:10356000300E822741EC0BF030C182F40401300EA2
:10357000822741EC0BF031C182F40401300E822726
:1035800041EC0BF004012E0E826F41EC0BF032C1C6
:1035900082F40401300E822741EC0BF033C182F437
:1035A0000401300E822741EC0BF004016D0E826F96
:1035B00041EC0BF01200120E2DEC09F0E8CF00F1F7
:1035C000130E2DEC09F0E8CF01F1140E2DEC09F0EB
:1035D000E8CF02F1150E2DEC09F0E8CF03F101015F
:1035E0000A0E046F000E056F000E066F000E076FC7
:1035F0002CEC20F0000E046F120E056F000E066F0B
:10360000000E076F4CEC20F0B9EC20F02AC182F4D8
:103610000401300E822741EC0BF02BC182F404012F
:10362000300E822741EC0BF02CC182F40401300EE5
:10363000822741EC0BF02DC182F40401300E822769
:1036400041EC0BF02EC182F40401300E822741ECD4
:103650000BF02FC182F40401300E822741EC0BF0F5
:1036600030C182F40401300E822741EC0BF00401DA
:103670002E0E826F41EC0BF031C182F40401300E4A
:10368000822741EC0BF032C182F40401300E822714
:1036900041EC0BF033C182F40401300E822741EC7F
:1036A0000BF00401730E826F41EC0BF012000A0E56
:1036B0002DEC09F0E8CF00F10B0E2DEC09F0E8CF6E
:1036C00001F10C0E2DEC09F0E8CF02F10D0E2DECFE
:1036D00009F0E8CF03F18CEF1BF0060E2DEC09F09A
:1036E000E8CF00F1070E2DEC09F0E8CF01F1080E4C
:1036F0002DEC09F0E8CF02F1090E2DEC09F0E8CF2E
:1037000003F18CEF1BF0010116EC21F0078457C187
:1037100000F158C101F107940101E80E046F800E19
:10372000056F000E066F000E076F2CEC20F0000EE8
:10373000046F040E056F000E066F000E076F4CEC51
:1037400020F0880E046F130E056F000E066F000E3A
:10375000076F1BEC20F00A0E046F000E056F000EC1
:10376000066F000E076F4CEC20F0B9EC20F0010161
:103770002967C0EF1BF00401200E826FC3EF1BF01E
:1037800004012D0E826F41EC0BF030C182F4040174
:10379000300E822741EC0BF031C182F40401300E6F
:1037A000822741EC0BF032C182F40401300E8227F3
:1037B00041EC0BF004012E0E826F41EC0BF033C193
:1037C00082F40401300E822741EC0BF00401430E19
:1037D000826F41EC0BF0120087C32AF188C32BF1F2
:1037E00089C32CF18AC32DF18BC32EF18CC32FF129
:1037F0008DC330F18EC331F190C332F191C333F1F7
:103800000101296B64EC21F0DBEC20F00101000EDA
:10381000046F000E056F010E066F000E076F2CEC93
:1038200020F00E0E0C6E00C10BF016EC09F00F0E1E
:103830000C6E01C10BF016EC09F0100E0C6E02C1FB
:103840000BF016EC09F0110E0C6E03C10BF016EC28
:1038500009F004017A0E826F41EC0BF004012C0E8A
:10386000826F41EC0BF00401350E826F41EC0BF0DE
:1038700004012C0E826F41EC0BF068EC1AF04FEF54
:1038800014F087C32AF188C32BF189C32CF18AC3B2
:103890002DF18BC32EF18CC32FF18DC330F18EC36C
:1038A00031F190C332F191C333F10101296B64EC22
:1038B00021F0DBEC20F0880E046F130E056F000E74
:1038C000066F000E076F20EC20F0000E046F040E50
:1038D000056F000E066F000E076F2CEC20F0010143
:1038E000E80E046F800E056F000E066F000E076F66
:1038F0004CEC20F00A0E0C6E00C10BF016EC09F037
:103900000B0E0C6E01C10BF016EC09F00C0E0C6ED8
:1039100002C10BF016EC09F00D0E0C6E03C10BF09A
:1039200016EC09F004017A0E826F41EC0BF00401F1
:103930002C0E826F41EC0BF00401360E826F41ECCD
:103940000BF004012C0E826F41EC0BF057EC1BF0D6
:103950004FEF14F087C32AF188C32BF189C32CF1F0
:103960008AC32DF18BC32EF18CC32FF18DC330F19F
:103970008FC331F190C332F191C333F1010164EC93
:1039800021F0DBEC20F0000E046F120E056F000E2C
:10399000066F000E076F2CEC20F001010A0E046F79
:1039A000000E056F000E066F000E076F4CEC20F046
:1039B000120E0C6E00C10BF016EC09F0130E0C6E1B
:1039C00001C10BF016EC09F0140E0C6E02C10BF0E5
:1039D00016EC09F0150E0C6E03C10BF016EC09F095
:1039E00004017A0E826F41EC0BF004012C0E826F01
:1039F00041EC0BF00401370E826F41EC0BF0040137
:103A00002C0E826F41EC0BF0DBEC1AF04FEF14F050
:103A100087C32AF188C32BF189C32CF18AC32DF106
:103A20008BC32EF18CC32FF18DC330F18EC331F1D6
:103A300090C332F191C333F10101296B64EC21F0A1
:103A4000DBEC20F0880E046F130E056F000E066F7E
:103A5000000E076F20EC20F0000E046F040E056FBF
:103A6000000E066F000E076F2CEC20F00101E80E2F
:103A7000046F800E056F000E066F000E076F4CEC92
:103A800020F0060E0C6E00C10BF016EC09F0070ECC
:103A90000C6E01C10BF016EC09F0080E0C6E02C1A1
:103AA0000BF016EC09F0090E0C6E03C10BF016ECCE
:103AB00009F004017A0E826F41EC0BF004012C0E28
:103AC000826F41EC0BF00401380E826F41EC0BF079
:103AD00004012C0E826F41EC0BF06DEC1BF04FEFEC
:103AE00014F007A8E4EF1DF00101800E006F1A0E1C
:103AF000016F060E026F000E036F4BC104F14CC143
:103B000005F14DC106F14EC107F11BEC20F003BFDA
:103B10002AEF1EF076EC1EF04BC100F14CC101F112
:103B20004DC102F14EC103F1078228EC1FF018C10C
:103B300004F119C105F11AC106F11BC107F1F80E14
:103B4000006FCD0E016F660E026F030E036F1BEC4C
:103B500020F00E0E0C6E00C10BF016EC09F00F0EEB
:103B60000C6E01C10BF016EC09F0100E0C6E02C1C8
:103B70000BF016EC09F0110E0C6E03C10BF016ECF5
:103B800009F00784010116EC21F057C100F158C17A
:103B900001F107940A0E0C6E00C10BF016EC09F04F
:103BA0000B0E0C6E01C10BF016EC09F00C0E0C6E36
:103BB00002C10BF016EC09F00D0E0C6E03C10BF0F8
:103BC00016EC09F02AEF1EF007AA2AEF1EF0078470
:103BD000010116EC21F057C100F158C101F1079421
:103BE000060E0C6E00C10BF016EC09F0070E0C6E01
:103BF00001C10BF016EC09F0080E0C6E02C10BF0BF
:103C000016EC09F0090E0C6E03C10BF016EC09F06E
:103C1000078462C100F163C101F164C102F165C1B1
:103C200003F10794120E0C6E00C10BF016EC09F0B4
:103C3000130E0C6E01C10BF016EC09F0140E0C6E95
:103C400002C10BF016EC09F0150E0C6E03C10BF05F
:103C500016EC09F00798079A0401805181197F0B2F
:103C60000DE09EA8FED714EE00F081517F0BE126F7
:103C7000E750812B0F01AD6E2CEF1EF093EF0AF091
:103C800018C100F119C101F11AC102F11BC103F100
:103C9000000E046F000E056F010E066F000E076F19
:103CA0004CEC20F029A16BEF1EF02051D8B46BEF43
:103CB0001EF018C100F119C101F11AC102F11BC1B6
:103CC00003F1000E046F000E056F0A0E066F000E62
:103CD000076F4CEC20F01200010104510013055154
:103CE0000113065102130751031312000101186B4F
:103CF000196B1A6B1B6B12002AC182F40401300E7F
:103D0000822741EC0BF02BC182F40401300E822794
:103D100041EC0BF02CC182F40401300E822741ECFF
:103D20000BF02DC182F40401300E822741EC0BF020
:103D30002EC182F40401300E822741EC0BF02FC11A
:103D400082F40401300E822741EC0BF030C182F482
:103D50000401300E822741EC0BF031C182F40401E2
:103D6000300E822741EC0BF032C182F40401300E98
:103D7000822741EC0BF033C182F40401300E82271C
:103D800041EC0BF012002FC182F40401300E8227A7
:103D900041EC0BF030C182F40401300E822741EC7B
:103DA0000BF031C182F40401300E822741EC0BF09C
:103DB00032C182F40401300E822741EC0BF033C192
:103DC00082F40401300E822741EC0BF01200060E43
:103DD0001F6E060E206E060E216E1F2EEDEF1EF0DA
:103DE000202EEDEF1EF0212EEDEF1EF08B84020E43
:103DF0001F6E020E206E020E216E1F2EFDEF1EF0B2
:103E0000202EFDEF1EF0212EFDEF1EF08B941200F0
:103E1000FF0E206E20C021F0030E1F6E8B841F2E1C
:103E20000EEF1FF0030E1F6E212E0EEF1FF08B946E
:103E300020C021F0030E1F6E1F2E1CEF1FF0030E7B
:103E40001F6E213E1CEF1FF0202E0AEF1FF0120004
:103E50000101005305E1015303E1025301E1002B8D
:103E6000EBEC1FF016EC21F03951006F3A51016F65
:103E7000420E046F4B0E056F000E066F000E076FAB
:103E80002CEC20F000C104F101C105F102C106F1E2
:103E900003C107F118C100F119C101F11AC102F102
:103EA0001BC103F107B259EF1FF020EC20F05BEFCC
:103EB0001FF01BEC20F000C118F101C119F102C183
:103EC0001AF103C11BF1120016EC21F059C100F1E7
:103ED0005AC101F1060E2DEC09F0E8CF04F1070EEE
:103EE0002DEC09F0E8CF05F1080E2DEC09F0E8CF34
:103EF00006F1090E2DEC09F0E8CF07F11BEC20F0DC
:103F000000C124F101C125F102C126F103C127F14D
:103F1000290E046F000E056F000E066F000E076F6E
:103F20002CEC20F0EE0E046F430E056F000E066FB2
:103F3000000E076F20EC20F024C104F125C105F12B
:103F400026C106F127C107F12CEC20F000C11CF1BD
:103F500001C11DF102C11EF103C11FF1120E2DECB2
:103F600009F0E8CF04F1130E2DEC09F0E8CF05F1CC
:103F7000140E2DEC09F0E8CF06F1150E2DEC09F02A
:103F8000E8CF07F10D0E006F000E016F000E026FFB
:103F9000000E036F2CEC20F0180E046F000E056F5E
:103FA000000E066F000E076F4CEC20F01CC104F1F0
:103FB0001DC105F11EC106F11FC107F120EC20F063
:103FC0006A0E046F2A0E056F000E066F000E076F53
:103FD0001BEC20F01200BF0EFA6E200E3A6F396B08
:103FE000D8900037013702370337D8B0FCEF1FF005
:103FF0003A2FF1EF1FF039073A070353D8B41200F4
:104000000331070B80093F6F03390F0B010F396F25
:1040100080EC5FF0406F390580EC5FF0405D405F01
:10402000396B3F33D8B0392739333FA911EF20F02E
:1040300040513927120001013BEC21F0D8B01200A9
:10404000010103510719346FFEEC20F0D89007519D
:10405000031934AF800F12000101346B22EC21F000
:10406000D8A038EC21F0D8B012000DEC21F016ECFD
:1040700021F01F0E366F4EEC21F00B35D8B0FEEC60
:1040800020F0D8A00335D8B01200362F3BEF20F037
:1040900034B125EC21F012000101346B04510511FB
:1040A000061107110008D8A022EC21F0D8A038ECA6
:1040B00021F0D8B01200086B096B0A6B0B6B4EEC49
:1040C00021F01F0E366F4EEC21F007510B5DD8A486
:1040D00076EF20F006510A5DD8A476EF20F0055166
:1040E000095DD8A476EF20F00451085DD8A089EFCF
:1040F00020F00451085F0551D8A0053D095F065125
:10410000D8A0063D0A5F0751D8A0073D0B5FD890A5
:104110000081362F63EF20F034B125EC21F0346BB1
:1041200022EC21F0D89052EC21F007510B5DD8A47D
:10413000A6EF20F006510A5DD8A4A6EF20F00551A5
:10414000095DD8A4A6EF20F00451085DD8A0B5EF12
:1041500020F0003FB5EF20F0013FB5EF20F0023F27
:10416000B5EF20F0032BD8B4120034B125EC21F0C8
:1041700012000101346B22EC21F0D8B0120057EC90
:1041800021F0200E366F003701370237033711EE6A
:1041900033F00A0E376FE7360A0EE75CD8B0E76EE9
:1041A000E552372FCBEF20F0362FC3EF20F034B19C
:1041B0002981D890120001010A0E346F200E366F4B
:1041C00011EE29F03451376F0A0ED890E652D8B06C
:1041D000E726E732372FE6EF20F0033302330133CF
:1041E0000033362FE0EF20F0E750FF0FD8A0033563
:1041F000D8B0120029B125EC21F01200045100279B
:104200000551D8B0053D01270651D8B0063D02271B
:104210000751D8B0073D032712000051086F015124
:10422000096F02510A6F03510B6F12000101006BFD
:10423000016B026B036B12000101046B056B066BD3
:10424000076B12000335D8A012000351800B001F2A
:10425000011F021F031F003F35EF21F0013F35EF23
:1042600021F0023F35EF21F0032B342B0325120000
:104270000735D8A012000751800B041F051F061F29
:10428000071F043F4BEF21F0053F4BEF21F0063FA6
:104290004BEF21F0072B342B072512000037013795
:1042A00002370337083709370A370B371200010185
:1042B000296B2A6B2B6B2C6B2D6B2E6B2F6B306B42
:1042C000316B326B336B120001012A510F0B2A6FD5
:1042D0002B510F0B2B6F2C510F0B2C6F2D510F0BE4
:1042E0002D6F2E510F0B2E6F2F510F0B2F6F305143
:1042F0000F0B306F31510F0B316F32510F0B326F8B
:0843000033510F0B336F120063
:10BF0000E844F926000C160C2B0C3F0C520C640C68
:10BF1000760C860C960CA50CB30CC10CCF0CDC0C6B
:06BF2000E80CF40C000C1B
:00000001FF
